:0200000480007A
:100000009710000093800000171100001301810178
:1000100083A1000013A2110093A2F17F13A3F1FFAB
:1000200093A3010013A40180232031002322410067
:10003000232451002326610023287100232A8100F4
:1000400097100000938040FC17110000130101FF7E
:1000500003A40000932414001325F47F9325F4FFD8
:10006000132604009326048023208100232291007C
:100070002324A1002326B1002328C100232AD10074
:1000800097100000938080F817110000130181FC85
:1000900083A6000013A7160093A7F67F13A8F6FF08
:1000A00093A8060013A906802320D1002322E10093
:1000B0002324F1002326010123281101232A2101F1
:1000C000971000009380C0F417110000130101FA8B
:1000D00003A9000093291900132AF97F932AF9FF35
:1000E000132B0900932B09802320210123223101A6
:1000F000232441012326510123286101232A710170
:1001000097100000938000F117110000130181F790
:1001100083AB000013AC1B0093ACFB7F13ADFBFF64
:1001200093AD0B0013AE0B802320710123228101BC
:10013000232491012326A1012328B101232AC101EF
:10014000171D0000130D4DED971D0000938D0DF54B
:1001500083200D0013A0100023A01D0023A20D007A
:10016000971F0000938F0FF4932010001321F07F4E
:100170009321F0FF132200009322008023A00F00A0
:1001800023A21F0023A42F0023A63F0023A84F0073
:1001900023AA5F00971F0000938F4FF29320100057
:1001A00013A11000132E1100932E1E0013AF1E007A
:1001B00023A00F0023A21F0023A42F0023A6CF01FA
:1001C00023A8DF0123AAEF0117150000130585E519
:1001D00097150000938505F0370610F01306C6F258
:1001E0006306B5028326C5002320D600832685003A
:1001F0002320D600832645002320D6008326050031
:100200002320D600130505016FF09FFD370510F080
:10021000130505F223200500000000000000000087
:0402200000000000DA
:101000000000000001000000FFFFFFFFFFFFFF7F67
:1010100000000080FFFFFFFF000000000000000054
:10102000FFFFFFFFFFFFFFFFFFFFFFFFFFFFFFFFD0
:10103000FFFFFFFFFFFFFFFFFFFFFFFFFFFFFFFFC0
:10104000FFFFFFFFFFFFFFFFFFFFFFFFFFFFFFFFB0
:10105000FFFFFFFFFFFFFFFFFFFFFFFFFFFFFFFFA0
:10106000FFFFFFFFFFFFFFFFFFFFFFFFFFFFFFFF90
:10107000FFFFFFFFFFFFFFFFFFFFFFFFFFFFFFFF80
:10108000FFFFFFFFFFFFFFFFFFFFFFFFFFFFFFFF70
:10109000FFFFFFFFFFFFFFFFFFFFFFFFFFFFFFFF60
:1010A000FFFFFFFFFFFFFFFFFFFFFFFFFFFFFFFF50
:1010B000FFFFFFFFFFFFFFFFFFFFFFFFFFFFFFFF40
:1010C000FFFFFFFFFFFFFFFFFFFFFFFFFFFFFFFF30
:040000058000000077
:00000001FF
